:030000000219FDE5
:03000B000200A848
:03002B000201547B
:03005B000202DAC4
:030073000202C7BF
:1000800002030406080C10182030406080040608A3
:100090000C10182030406080A0C00003070F1F051F
:1000A000050D050205030302C2AFC0D0C0E0206207
:1000B00014E5256009E473E525F4F58AD262D0E001
:1000C000D0D0D2AF3285268AC262E526F46029D02C
:1000D000E0D0D0C293C295C297D2AF32C293C2953C
:1000E000C297206F0C206509740ED5E0FDE57B42B8
:1000F00090D0E0D0D0D2AF32758A00C28DD26201EA
:10010000F101B7306805206502D29301B730680568
:10011000206502D29501B7306805206502D29701AB
:10012000B7C29230680A206507740CD5E0FDD293FF
:1001300001B7C29430680A206507740CD5E0FDD27F
:100140009501B7C29630680A206507740CD5E0FDAA
:10015000D29701B7C2AFC2AD53E6EFC0D0C0E0D274
:10016000D3D2AFC2CEE52A600720744F152A21BB37
:100170007800790020742EE580307E01F430E302AF
:1001800078FF53DACF207E0343DA20307E0343DA50
:1001900010C2D8C271E580307E01F430E30279FFED
:1001A000C3E89970CB306103752A18207403752A4F
:1001B00018885CD270E86003755F0020740DE52B31
:1001C0006004152B21CB43DA01C2D8207002413ED6
:1001D000A85C206102C270207431C3E894F040032F
:1001E00074F0F8E8C4540F28F87984B70302410B7F
:1001F000C313C3138721200802C313200A06C3C8F0
:1002000098F8410B28F8500374FFF8C3E89565503F
:1002100003E565F88822E52D54066022206B1FE572
:1002200036C333C333F8E564C313C313F9C395224C
:1002300040028922E82522F52250037522FF8522FB
:1002400024A824C3E52495614002A8618825E566B9
:1002500070024182C3E8AA669A5003E8FAE4F9EA18
:10026000C333FBE568F45B29400D2567F8E567605B
:10027000021567400B41820AC3E5679A5002056781
:1002800078FF882620CF0AD0E0D0D043E610D2AD48
:1002900032C2CF053A7801E52A6005307402152A8A
:1002A000C3E55C94014005755F0041BD7560007554
:1002B0006900E55F2401F55F5003755FFFD0E0D072
:1002C000D043E610D2AD32C2AF53E67F7592FA75D5
:1002D00093FFC260759104D2AF32C2AF53E6EFC252
:1002E000ADC0D0C0E0C0F0D2D3D2AFA8FBA9FCC251
:1002F000D8307102614153DACF207E0343DA1030E7
:100300007E0343DA20D271E580307E01F420E302DF
:10031000611888278928A16E53DACF207E0343DA3B
:1003200020307E0343DA10C2D8C271307402A15A61
:100330007800E580307E01F430E302A15A885CA1A8
:100340004253DACF207E0343DA20307E0343DA10B3
:10035000C271206102811A53DACF207E0343DA1082
:10036000307E0343DA20C2D8D27188578958C3E857
:100370009555F8E99556F97B007E087A00C3E89414
:100380008CE994005005755B00810C882178A2E609
:10039000A8216055C3E894C8E994005008E4D2E469
:1003A000FB7A0A61E7C3E89468E994015008E4D253
:1003B000E3FB7A0F61E7C3E894D0E994025008E4C4
:1003C000D2E2FB7A1E61E7C3E894A0E994055008E5
:1003D000E4D2E1FB7A3C61E7C3E89498E9940850E1
:1003E00008E4D2E0FB7A787E00C3E89559FCE995F1
:1003F0005AFD30E70AECF42401FCEDF43400FD75FD
:100400005B00C3EC9AED9E5003755B018859895AD5
:100410008557558558567802A142C3E89527F8E9D3
:100420009528F9307C02A126307B02A126307A0281
:10043000A11F207502813DE9FDE8FC815CE9C31341
:10044000F9E813F8307902A11FE9C313F9E813F8AA
:10045000307802A11FE9C313FDE813FC20612CC30F
:10046000EC941CED940240028173ED701EC3EC9479
:0E047000C850180529E52970021529C3E52991
:10047E00940A5002A15A755C00D270A15AE5296007
:10048E000215297888E6F97400207F087896B9035A
:10049E0002789EE624FAFEE43400FFC3EC9EFCEDE7
:1004AE009FFD9208B90310A2085007207609D27654
:1004BE0081C5307602C276A2085016B9030DECF44F
:1004CE002401FCEDF43400FD0204DF78007900A174
:1004DE0026B90315EC33FCED33FDC3EC940AFCEDA9
:1004EE009400FD50047C007D00C3EC94FFED94005D
:1004FE00400678FF7900A126EC8572F0A4C5F0A223
:10050E00F733F87900400302054278FF79000205BF
:10051E0042E9C313F9E813F8307C0EE9600278FF64
:10052E00C3E81338F8E43400F9C3E894FFE9940003
:10053E00400278FF885CD270206102A15A741FF4C9
:10054E00552F4BF52FC274EB7002D274752A1830EA
:10055E007403752A0A306102A16E20740353DAFE09
:10056E00207403752B06D0F0D0E0D0D0D2AD43E688
:10057E001032790102059E790302059E790A020561
:10058E009E791E02059E796402059E79C802059E1B
:10059E007817E4D5E0FDD8FAD9F6227A147B7802E2
:1005AE0005C57A107B8C0205C57A0D7BB40205C594
:1005BE007A0B7BC80205C5E573D5E001227902E40A
:1005CE00C294D5E0FDD295D5E0FDC295D5E0FDD221
:1005DE0094D5E0FDE920E002D29330E002D297E517
:1005EE0073D5E0FDE920E002C29330E002C29774B9
:1005FE0096D5E0FDD9C9EAF8D5E0FDD8FBDBB8C247
:10060E009422C37C007D0075F00005F0EA33FAEB0E
:10061E0033FB50F6EB13FBEA13FAC3E9FFE8FEE8EF
:10062E009AF8E99BF95004EFF9EEF8B3EC33FCEDD0
:10063E0033FDD5F0DFEDF9ECF822E889F08A20D20F
:10064E00D4F8A9F07B0030F70B7BFFF42401F8E916
:10065E00F43400F9E88520F0A4ADF0F8E98520F037
:10066E00A4AFF0FEED2EF974003FFA7C04C3EA133A
:10067E00FAE913F9E813F8DCF48BF030F70AE8F432
:10068E002401F8E9F43400F9E889F0C2D4F8A9F0AD
:10069E002222C3E54113F9E54013F8C3E54498F867
:1006AE00E54599F9500CC3E89480E994FF40160291
:1006BE0006D7C3E8947FE9940050030206D7787FEB
:1006CE0079000206D7788079FF8849894A22E54960
:1006DE002546F8E54A3547F9854A20E4300701F406
:1006EE003548FA30E709C3EA94F04015020715C3FE
:1006FE00EA940F500302071578FF79FF7A0F02076D
:10070E0015780079007AF0C3E5249561500AC37418
:10071E00019524500B020733E54A20E70E020733FA
:10072E00E54A30E706884689478A482278A5E6FAE0
:10073E00C3E54933F8E54A33F9D148E930E70BC34D
:10074E00E89480E994FF4013E16DC3E8947FE99447
:10075E00005002E16D787F7900E16D788079FFE8D5
:10076E0020E715C3E52398F84009C3E89401400338
:10077E000207947801020794E8F424012523F84037
:10078E000302079478FF884B2278A6E6FAA847A9B9
:10079E0048D148E930E70CC3E89401E994FF4016CC
:1007AE000207C8C3E894FFE9940050030207C87813
:1007BE00FF79000207C8780179FFE920E715C3E544
:1007CE004B98F84009C3E8940140030207EF780103
:1007DE000207EFE8F42401254BF840030207EF78F7
:1007EE00FF88242278FF20692879A1E76023E5415C
:1007FE00601F74FF8541F0848539F0306A0375F00F
:10080E0005A4F8C5F0600278FFC3E895645002A80D
:10081E0064886322C3E5409440E5419401E563504A
:10082E0003140133046002F5632202083B2275E8CB
:10083E0090227883E6FF30EDF9A8BDA9BE0570C3FE
:10084E00E57094084052757000E9FA79A0E76044AB
:10085E00EA7007E571601B020874C3E895716010B9
:0D086E00E5715006600C140208800460F96A
:10087B00020880E571F571C394A8401B7561C0C374
:10088B0094054013756180C39405400B756140C39B
:10089B009405400375610075BB0122E561F46002AC
:1008AB000561E570B4070375BB1E22743279A78707
:1008BB00F0A4C5F0A2F733F8C3E895614002A86134
:1008CB0088228824882588268864227540007541F3
:1008DB00F022C2AF75C820A8CCA9CDAA3A30CF015F
:1008EB000A75C824D2AFAB3BAC3C883B893CC3E810
:1008FB009BF8E99C206908F930660221EE2148AD8E
:10090B003D8A3DF9EA9DFA600678FF79FF212DAE0D
:10091B003EAF3F8B3E8C3FA83BA93CC3E89EF8E91A
:10092B009FF9C3E54113FBE54013FAE82AF540E9CB
:10093B003BF54150067540FF7541FF2195AA40AB31
:10094B0041AC40AD417E047F02C3EB9404400D1ECD
:10095B001FC3EB94084005206A021E1FC3ED13FD55
:10096B00EC13FCDEF7C3EA9CFAEB9DFBEF6009C3CB
:10097B00E913F9E813F8DFF7EA28FAEB39FB8A40B9
:10098B008B4150067BFF8B408B41C3EB9402500293
:10099B00D2663069047F0321C07892E6FFC3E53746
:1009AB00948240110FC3E53794A040010FC3EF941D
:1009BB000640027F057E02E541C4540FF9E541C4B0
:1009CB0054F0F8E540C4540F28F8C3E89EFAE994B4
:1009DB0000FB4009C3EA9402EB940050047A02E452
:1009EB00FB413AAA40AB41EBC4FEEAC4540F4EFCA8
:1009FB00C3EA9CFAEB9400FBC3E813C313F8EA2891
:100A0B00FAEB3400FB8A408B41C3EB94024002C2E9
:100A1B00667802EBC4FE7B00EAC4540F4EFAC3EABD
:100A2B0098FA4005C3940250027A027892E6FF309E
:100A3B006002413A855192855293D26043E680C35E
:100A4B00E49AF8E49BF930660241C6E8FAE9FBD375
:100A5B00E913FDE813FC88518952C3EF9403603806
:100A6B00EF20E00DE82CF8E93DF9ECFAEDFB020A7A
:100A7B008FE828F8E939F9C3E82402F8E93400F9DA
:100A8B007AFE7BFFC3EF9403400E8A538B54884D41
:100A9B00894E8C4F8D5041FA885389548A4D8B4E19
:100AAB008C4F8D503069127553F07554FF754FF0A4
:100ABB007550FF7551F07552FF41FAE8FAD3E81300
:100ACB00FC8851C3EF94036020EF20E007E82CF87B
:100ADB00ECFA41E6E8282402F87AFEC3EF940340CF
:100AEB00088A53884D8C4F41FA88538A4D8C4FE5B9
:100AFB0068C3335002646BF568306002610475346F
:100B0B0002D26043E680E52D54066034A840A9412B
:100B1B00C3E913F9E813F8C3E913F9E813F83069DB
:100B2B0004E92440F9C2AF53E67F759100C3E49802
:100B3B00F594E499F595759104D26043E680D2AFB4
:100B4B0022D264754300752000306C03752040027F
:100B5B000B6BD264754300752040306C037520001D
:100B6B0078017901206620E52D54066002C2647974
:100B7B0014E541C313700104F8C3941440027814B4
:100B8B00306904781B791B206010E543600C3069D9
:100B9B0003D53404D26D811E710C0543E59E70059F
:100BAB00E59B020BB2E59A5440B5200281083069EF
:100BBB000908C3E899400118619220640A08C3E848
:100BCB00994002616B6192C264C2AF53E67F75912B
:100BDB00003066127594007595F8759104D26043D8
:100BEB00E680D2AF616BE5417EFFC3334005C33373
:100BFB004001FEC3E49E759400F59561E5C3E533B2
:100C0B0094015002616B306402616BD802811C61EC
:100C1B0092C26DC2AF53E67F759100855394855494
:100C2B0095759104854D92854E93D26043E680D2A3
:100C3B00AFE52D54066008206A020533020C5A30CA
:100C4B006D0D206C0A2064071581158102154B224E
:100C5B0078003064027801E53775F007A4F9E5F008
:0F0C6B0028F5F0E9A2F013A2F113A2F213F53766
:100C7A00C394785003753778C3E53795384008D25E
:100C8A0065C293C295C2973060028191854F928561
:100C9A005093D26043E68022207D19C2AF7542028A
:100CAA00C294D292306202D297D2AF759F33759EA8
:100CBA0000020EA4C2AF754202C294D296306202FA
:100CCA00D293D2AF759F33759E00020EA430724341
:100CDA00207D20C2AF754203900132757B10C29706
:100CEA00C296306204D29581F5D294D2AF759E2312
:100CFA00020EA4C2AF754203900132757B10C293F3
:100D0A00C292306204D295A115D294D2AF759E22B6
:100D1A00020EA4207D17C2AF75420390010DC2973F
:100D2A00306202D295D2AF759E23020EA4C2AF756D
:100D3A00420390010DC293306202D295D2AF759EE2
:100D4A0022020EA4207D16C2AF754204C292D29628
:100D5A00306202D295D2AF759E22020EA4C2AF753E
:100D6A004204C296D292306202D295D2AF759E23C5
:100D7A00020EA4307249207D23C2AF75420590014C
:100D8A0021757B04C295C294306204D293A19BD28E
:100D9A0092D2AF759F33759E00020EA4C2AF754200
:100DAA0005900143757B40C295C294306204D29784
:100DBA00A1BED296D2AF759F33759E00020EA420B3
:100DCA007D1AC2AF754205900103C295306202D204
:100DDA0093D2AF759F33759E00020EA4C2AF7542BF
:100DEA0005900117C2953062E8D297D2AF759F334A
:100DFA00759E00020EA4207D16C2AF754206C296E9
:100E0A00D294306202D293D2AF759E23020EA4C24C
:100E1A00AF754206C292D294306202D297D2AF75AF
:100E2A009E22020EA4307244207D20C2AF75420178
:100E3A00900143757B40C293C292306204D297C13B
:100E4A004DD296D2AF759E22020EA4C2AF75420150
:100E5A00900121757B04C297C296306205D2930233
:100E6A000E6ED292D2AF759E23020EA4207D17C2B7
:100E7A00AF754201900117C293306202D297D2AF86
:100E8A00759E22020EA4C2AF754201900103C29759
:100E9A00306202D293D2AF759E23C26522900101BD
:100EAA00757B00C293C295C297C292C294C296C27F
:100EBA006222788076FF0876FF0876FF0876FF08B8
:100ECA00760308760408760708760108760108761C
:100EDA0001788C76010876FF0876FF0876FF087697
:100EEA00FF0876FF0876030876FF0876FF0876FF84
:100EFA000876250876D00876FA0876FA087604087D
:100F0A0076FF08760108760008767A0876FF087672
:100F1A0001087601087600087603087600227887A9
:100F2A00E6FFC2727888E6C394036008C27DE630A1
:100F3A00E102D27DC27E7889E630E102D27EC3EF39
:100F4A0094026008758E01D273020F5B758E00C21F
:100F5A0073227880E6149000809378A5F67881E66B
:100F6A00149000809378A6F67886E61490008D9304
:100F7A0078A7F67886E6F539C394025003753902E4
:100F8A00789CE67538FFB402037538A0B40303757C
:100F9A00388278A3E61490009A93F566D1A72222A4
:100FAA007896E6FA7897E6FB7888E6B40305C3EB09
:100FBA00940EFB307F047A007BFFC3EB9AFCC39448
:100FCA008250027C827572000572EC8572F0A4C3AD
:100FDA00E5F0947D40F222D27FF1AA12058F120524
:100FEA008F7A007B007C10120585E55C2AFA740072
:100FFA003BFBDCF37C04C3EB13FBEA13FADCF7FEDE
:10100A00C27F120FAA22757C00757D00E5EF20E6EB
:10101A00037520000520903DFFE520146006901F0F
:10102A00FF1460009304600375EF1653D9BF7581EE
:10103A00C043FF8012058075EF0643B203E5B3246F
:10104A000220E70DF521E5B120E0068521B343B181
:10105A0001120EA77580FF75A40075F1FE75D4F70D
:0F106A0075900275A5FC75F2FC75D50075A0FD9B
:1010790075A60275F30275D60075B0FF75A70175DF
:10108900F4FF75E241120EA7E4F8F6D8FD75680180
:10109900120EBC12159C78988673753001C2AF1276
:1010A90005991205A912058F1205B012058F1205AF
:1010B900B712058F1216C5120599120599120594D2
:1010C900C2AF757C00757D0078FA79FA308307D94B
:1010D900FBD8F7021C00120F28120F5C120FA9127D
:1010E9000FAA78988673120EA775881075890275EC
:1010F900C82475910475D84075A82275B80275E69B
:1011090090759B80759D00759A80759C0075D10EB0
:1011190075BC5875BB0175BA1F75E880120580D278
:10112900AF12083875360053DACF207E0343DA2030
:10113900307E0343DA1043DA01C2D8C2711205992D
:10114900D2617B037A0CE55B70077A0CDB03021032
:10115900C912058F2070030210C9C270E55CC394DF
:101169000240E1E52F541F855E5DF55EB55DD5DA78
:10117900D5C26153DACF207E0343DA20307E0343A0
:10118900DA10C2D8C27178A2E67008D274E52F5479
:10119900E0F52FC275752900120594307409C3E56D
:1011A90029940A4002D275120585780230740278B2
:1011B90000C3E55C9840F0C2AF1205A91205A91257
:1011C90005A9D2AF120599754C007888E6B40302D7
:1011D90041CF120585788CE6C3940150030212CFE2
:1011E900E530C3940150030212CF757CA5757DF1DA
:1011F900207435C3E55C94FF50030212CFC2AF12CD
:1012090005BED2AF120594C3E55C940150EFC2AF9D
:101219001205A912058A1205A9D2AF120594C3E5D0
:101229005C94FF40E902174A7F05D27F120FAA1288
:101239000594C2AFC27F120FAAAE5CC3E55C947F6E
:10124900D2AF500241DF120580C2AF1205BED2AF44
:10125900DFD8120FE1C3EE94057897F612059912BB
:1012690016CD7F0AD27F120FAA120594C2AFC27F90
:10127900120FAAAE5CC3E55C947FD2AF50E41205AD
:1012890080C2AF1205A912058A1205A9D2AFDFD40F
:10129900120FE1EE24037896F6F87997E7C3948262
:1012A9004003985006E824827897F612059912159A
:1012B900EA1216FC120594120FAAC3E55C94FF50BA
:1012C9000221F302174A757C00757D00C3E55C9520
:1012D9004C4003855C4C12059478017988E7B40386
:1012E900027805C3E55C98400221D3C2AF1205BE5E
:1012F9001205BE1205BED2AF120599753000E4F58C
:1013090031F5320531E531F4703F0532789AE678E6
:1013190019146012783214600D787D14600878FA17
:10132900146003753200C3E53298401D120EA712EE
:101339000580153275310078998673C2AF1205BEE2
:10134900D2AF7898867312059412058AE52A70053A
:1013590030740201C978012074027806C3E55C98EB
:1013690040A17888E6C394036003120594E52A70C6
:10137900030210C9C2AF120EA7E4F522F523F52422
:10138900F525F526F567D2AF7885E6C333F565E42B
:10139900F544F545F546F547F548F570F52CF52D75
:1013A900F53775700875BB1E12058012083C30EDC3
:1013B900FDA8BDA9BEE97001F888711208407570D1
:1013C9000875BB1E120F28C2AF7561FF1208B685DA
:1013D9002261852262852263D2AF752201752401BB
:1013E900752501752601856069756A017888E6B4F5
:1013F9000307C27D307602D27DD268D26975330087
:10140900120E00120E2F1208D61208DD1208D6127B
:1014190008DD1208D6120B5D12069F120C5B120C26
:10142900A21208DD120B4C306E031206A0206603CF
:101439001207F2306603120822120C5B120CD71243
:1014490008DD120B5D306E031206DC120C5B120D07
:101459004E1208DD120B4C306E0312073A120C5B68
:0F146900120D7D1208DD120B5D306E0312079716
:10147800120C5B120E001208DD12083C120B4C1203
:101488000C5B120E2F1208401208DD30692F85649C
:1014980061856462856069756A0179187A0CC3E5AB
:1014A8003399400CC269D26A8A357561FF0214C546
:1014B800C3E55C9401400302141E021553306A25EB
:1014C800206C22E535147006C26AD26B811EF53590
:1014D800C3E55C9401400302141E7888E6C39403B4
:1014E8006003021553753600788279A4E7600278A4
:1014F80003C3E55F985054307404E52A604D78883A
:10150800E6B40317207D05207607A123307602A1D3
:1015180023206C07D26C856461815D78F0306C059E
:101528008564617820C3E541985002811E306C1BA8
:10153800C26CC27D307602D27DD26A75351285645E
:1015480061811E0536E55C6002A156753600C2AFA2
:10155800120EA77887E6FE7602120F287887EEF635
:10156800E4F522F523F524F525F526F565752C0017
:10157800752D00D2AF120594120EA778A4E6600666
:10158800D293D295D297307409C3E53694044002B9
:1015980001C96107901A0D782012162CE520B45A5B
:1015A8000CA312162CE520B4A5030215CA757CA558
:1015B800757DF1120EBC1215EA757C00757D00026E
:1015C80015E9901A0378807B0A12162CA308DBF918
:1015D800901A0F788C7B1912162CA308DBF9901A35
:1015E8002822C2AF12166F12164C901A00740E12EF
:1015F8001631A37409121631A37415121631901AF4
:101608000378807B0A121630A308DBF9901A0F784A
:101618008C7B19121630A308DBF912168212166099
:10162800901A2822E493F622E6438F01538FFDFF98
:10163800C3E583941C400122EF857CB7857DB7F014
:10164800538FFE22438F02438F01857CB7857DB778
:10165800901A0DF0538FFC22901A0D745AD13190C4
:101668001A0E74A5D131227A3079D07820901A4098
:10167800D12CE520F709A3DAF7227A3079D0901A2D
:1016880040E7D13109A3DAF922AB74A875BB01028E
:101698007984BB02027985BB03027986BB0402798F
:1016A80092BB05027987BB060279A3BB0702799C26
:1016B800BB08027988BB09027989E8F7227C051200
:1016C8000599DCFB22C2AF1205A91205B01205B7B5
:1016D8001205BE12058A1205A91205B01205B71225
:1016E80005BE12058A1205A91205B01205B7120522
:1016F800BED2AF22C2AF1205BE1205B71205B01294
:1017080005A912058A1205BE1205B71205B0120501
:10171800A912058A1205BE1205B71205B01205A94D
:10172800D2AF22AE74AF75C2AF1205A91205A912C5
:1017380005A912058ADEF21205BE12058ADFF8D263
:10174800AF22D1CDD1C5D1C5757401757501757636
:1017580000F12B7C05AD5C120599C3ED955C70F525
:10176800C3E55C9401400AC3E55C94FF403202176C
:1017780086D191B1EAD1CDC2AF75EF16D1C5DCD50E
:101788000576C3E5769403500280C6D1C50575E594
:10179800741490009F93F808C3E57598500280AEC2
:1017A800D1C5D1C50574C3E574940A5002809C1252
:0B17B8000EBCB1EAC2AF75EF16D1C540
:0319FD00021010C5
:101A00000E0915FFFFFFFF0304070101015AA5019D
:101A1000FFFFFFFFFF03FFFFFF25D0FAFA04FF01DE
:091A2000007AFF0101000300FF40
:101A4000235467794B4631323041485623202020B9
:101A500023424C48454C4923463331302320202033
:101A60002020202020202020202020202020202076
:101C0000C2AFC2D353D9BF7581C043B20343FF8073
:101C1000752438752503B1DC7529A5752AF175E29F
:101C20004043F10853A4F775D4FFD2837DFA7803BB
:101C300079E67C10752200752300901DE97B0675FE
:101C400024987525013083028145208308D8FBD96B
:101C5000F9DCF781B7308308D8FBD9F9DCF781B715
:101C6000B19CE493A3C39A6004DDC381B7DBDBB10D
:101C70008E6002812E7B08E493FAA3B16FDBF87AC1
:101C800030B16F752200752300B18EEAFCEBFDC305
:101C9000ED94FE400EB18E8A278B28ED30E0048A49
:101CA000828B83B18E7AC270D8C3ED94FE601950D6
:101CB000CEBD002BEC600F7520007521FF7529004B
:101CC000752A000200008100A827A9280809D80465
:101CD000D90281DCB192EA89AAF281CE0D81A3C337
:101CE000ED94035053EDA2E092007AC5C3E58294CF
:101CF00000E583941C508A200010438F02438F011B
:101D00008529B7852AB7F0300029A827A92808090E
:101D1000438F01538FFDD804D902A133C3E58394C7
:101D20001C4003A3A11689AAE28529B7852AB7F02A
:101D3000A3A116538FFC817F7AC1BD030CE493A34A
:101D4000FAB153DCF8B14B817F8181AA22AB23B178
:101D50006FEBFAEA6222752608C3E52313F523E543
:101D60002213F52250066323A0632201D526EAB18F
:101D7000DCB1DC75260AEAF4200102D283300102CC
:101D8000C283B1DCC3134002C201D526EB22B1925B
:101D9000EAFB208302A192308302A197752608AE48
:101DA00024AF25C3EF13FFEE13FEB1E0B1DCC3EAAD
:101DB000133083024480FA30E703632201C3E52332
:101DC00013F523E52213F52250066323A0632201B5
:101DD000D526D9E52265236523F52222AE24AF2539
:101DE0000E0FDEFEDFFCD20122424C48656C6934E6
:071DF000373164F310060116
:00000001FF
